:100000000C9437010C9454010C9454010C94540139
:100010000C9454010C9454010C9454010C9454010C
:100020000C9454010C9454010C9454010C945401FC
:100030000C9424130C9454010C9454010C9454010A
:100040000C9454010C94FB050C94471B0C94331234
:100050000C94C3120C9454010C9454010C9454014C
:100060000C9454010C9454010C9454010C945401BC
:100070004570692D4F5344205665722E302E392E0F
:10008000352E320000416B7475656C6C65732053BE
:10009000657474696E67000053657474696E6720D7
:1000A000200000486F6568656E73656E736F72201F
:1000B00000004853206D697420536368616C746557
:1000C0007220000048656164696E6720486F6C6447
:1000D0002000004B6F6D706173732000004B6F6DDB
:1000E0007061737320666978200000475053204187
:1000F0006B74697620000041636873656E6B6F7086
:1001000070656C756E67200000447265687261747A
:100110006520626567722E2000004665686C657216
:100120002046433C2D3E4F5344200000556E7465DD
:10013000727370616E6E756E672000004B65696E3C
:10014000652053657474696E672D416E7A656967C1
:1001500065000050432F425420616B7469760000A3
:1001600055656265726E65686D65204C65747A745C
:1001700065732053657474696E6700004B65696E22
:1001800065204465766976652D416E7A6569676597
:10019000000050432F425420616B74697600005573
:1001A000656265726E65686D65204C65747A74650C
:1001B000732044657669636500004F4E00002D2D65
:1001C0002D000044657669636520756E6420566570
:1001D0007273696F6E736162667261676500004475
:1001E000657669636520202020203D200000465769
:1001F0002D56657273696F6E203D200000464300E6
:10020000004E43000046432D6F6C642046570000AB
:100210004550492D4D656E750050616C0050432F5F
:100220004254004B656E6E756E670052432D4265F9
:100230007472696562004550492D5374726F6D0088
:1002400045786974004F4E002D2D0076767D7676C8
:100250007A76767E76767776767B76767876767C24
:1002600076767976767D76767A76767E7600112445
:100270001FBECFEFD4E0DEBFCDBF11E0A0E0B1E004
:10028000E6E1F9E302C005900D92A239B107D9F772
:1002900013E0A2E9B1E001C01D92A43FB107E1F76C
:1002A0000E9464010C94891C0C94000086E981BBB7
:1002B0008FE084BBAC9AAD9A8EE28ABB80EB87BBA1
:1002C000C69AD99ADD9A08951092DA011092D60151
:1002D0001092DB01E199FECF80E090E09FBB8EBBE6
:1002E000E09A8DB380939901E199FECF81E090E08F
:1002F0009FBB8EBBE09A8DB380930001E199FECF46
:1003000082E090E09FBB8EBBE09A8DB380939A0110
:10031000E199FECF87E190E09FBB8EBBE09A8DB361
:100320008093A701E199FECF88E190E09FBB8EBB4F
:10033000E09A8DB38093C001E199FECF8AE190E00D
:100340009FBB8EBBE09A8DB380930901E199FECFEC
:1003500089E190E09FBB8EBBE09A8DB38093BC0196
:10036000E199FECF8BE190E09FBB8EBBE09A8DB30D
:1003700080939B0120910001213079F49EE09093BD
:10038000030187E08093040186E8809305012093B0
:100390000601909307018CE00EC09CE0909303014E
:1003A00085E0809304018AE48093050110920601A0
:1003B000909307018AE0809308010E9441180E94EF
:1003C00056010E94F40580919901813019F40E9430
:1003D0000E1102C00E94FE107894A89A0E941A057D
:1003E0000E945B060E944E0A80919B01882311F0B7
:1003F0000E948E0A8091C501882311F00E94341456
:100400000E948E0A80919B01813011F40E94971BFB
:100410000E94DF118091B801813021F41092B8015F
:100420000E94D9188091DF01813021F41092DF0100
:100430000E94240E809194018130C9F4109294019D
:100440008091DA01882369F48091BC01843049F4F9
:1004500080919901882329F480E364E641E00E94B9
:100460008D110E9417130E941C130E948415809105
:100470009B01813031F48091E001813011F40E94C0
:10048000A21B809197018130E1F48091DA018823E9
:10049000C1F4AA9A0E94650F0E94AE090E94C30887
:1004A0008091C301882321F00E9490130E940C0BBD
:1004B0008091C401882311F00E9489180E94E30AE8
:1004C000AA9880919201813009F03FC08091DA01B1
:1004D0008823D9F5109292018091BC01823029F4D1
:1004E00083E66FE64AE00E948D118091BC01813065
:1004F00029F482E664E64AE00E948D118091A7010A
:10050000882321F080910201833014F00E94BD0AFB
:100510008091A4019091A50101969093A5018093EB
:10052000A4010197CB9769F48091A2019091A30156
:1005300001969093A3018093A2011092A5011092BD
:10054000A4010E949C0C0E94E60D809193018130D1
:1005500009F060CF8091DA01882309F05BCF109217
:10056000930180919B01813039F48091E0018823CF
:1005700019F481E00E94A21B0E94570A8091C501D4
:10058000882309F447CF0E9490140E9410140E94FF
:10059000FB140E9461140E943C140E94F2133ACF93
:1005A000782FD99827E030E041E050E0DB98000058
:1005B000000000000000CA01022E02C0880F991F2F
:1005C0000A94E2F7872311F0DA9A01C0DA98000062
:1005D000000000000000DB9A0000000000000000A6
:1005E000215030408FEF2F3F380701F727E030E0F0
:1005F00041E050E0DB980000000000000000CA016C
:10060000022E02C0880F991F0A94E2F7862311F088
:10061000DA9A01C0DA980000000000000000DB9ABE
:100620000000000000000000215030408FEF2F3FFD
:10063000380701F7DB98DA98D99A089584E064E0E6
:100640000E94D00280E06CE40E94D00210929401DB
:10065000809194018823E1F38CE66AE00E94D00245
:1006600085E060E00E94D00208950F931F9380916F
:1006700092018823E1F3109292018091BC018230B3
:1006800051F40E941E1110929201809192018823D0
:10069000E1F3109292011092C2010E94650F82E66E
:1006A00061E74FEF0E948D1110E000E01DC08091C6
:1006B0009701813071F480917B02813519F40E9499
:1006C000650F02C08091970182E661E74FEF0E94BB
:1006D0008D1180919201813039F410E0023009F4DB
:1006E00011E0109292010F5F8091C201882311F4F2
:1006F0001123E9F28091BC01823011F40E9465114E
:10070000112309F0D9C08091E303809309018091FE
:10071000CD038093C0012091C001E199FECF88E113
:1007200090E09FBB8EBB2DBB0FB6F894E29AE19A86
:100730000FBE20910901E199FECF8AE190E09FBBB5
:100740008EBB2DBB0FB6F894E29AE19A0FBE82E001
:1007500061E045E850E00E94A00E82E062E048E9D6
:1007600050E00E94A00E82E064E043EA50E00E9464
:10077000A00E82E065E042EB50E00E94A00E82E015
:1007800066E044EC50E00E94A00E82E067E043ED9A
:1007900050E00E94A00E82E068E04DED50E00E9423
:1007A000A00E82E069E04BEE50E00E94A00E82E0D5
:1007B0006AE047EF50E00E94A00E82E06BE04CE25E
:1007C00051E00E94A00E4091BE015091BF0184E112
:1007D00062E00E94F90D8091C00180FF05C084E1B4
:1007E00064E04AEB51E004C084E164E04EEB51E088
:1007F0000E94A00E8091C00181FF05C084E165E0E8
:100800004AEB51E004C084E165E04EEB51E00E9408
:10081000A00E8091C00182FF05C084E166E04AEB32
:1008200051E004C084E166E04EEB51E00E94A00E6E
:100830008091C00183FF05C084E167E04AEB51E08D
:1008400004C084E167E04EEB51E00E94A00E80916D
:10085000C00184FF05C084E168E04AEB51E004C0B8
:1008600084E168E04EEB51E00E94A00E8091C0014F
:1008700085FF05C084E169E04AEB51E004C084E1F2
:1008800069E04EEB51E00E94A00E8091C00186FF0E
:1008900005C084E16AE04AEB51E004C084E16AE00B
:1008A0004EEB51E00E94A00E4091090184E16BE003
:1008B00050E00E94F90D20C082E062E045E850E07F
:1008C0000E94A00E82E065E04AE151E00E94A00E85
:1008D000E199FECF88E190E09FBB8EBBE09A8DB39B
:1008E0008093C903E199FECF8AE190E09FBB8EBB64
:1008F000E09A8DB3809309019091C903892F81708B
:100900008093C301892F88708093C401892F8072DE
:100910008093C50194709093C6011F910F91089523
:100920001F93809192018823E1F3109292018091AC
:1009300092018823E1F31092920183E666E740E09A
:100940000E948D1110E00DC080919701813011F44B
:100950000E94480F80919201813019F41092920107
:1009600011E08091BD01882311F4112369F3112353
:1009700009F054C082E062E043EC51E00E94A00E16
:1009800082E064E04FED51E00E94A00E82E066E05C
:100990004EEE51E00E94A00E8091BC01813031F4F6
:1009A0008EE064E04DEF51E00E94A00E8091BC010A
:1009B000823031F48EE064E041E052E00E94A00E0B
:1009C0008091BC01843031F48EE064E045E052E077
:1009D0000E94A00E409183038EE066E050E00E94EA
:1009E000F90D4091840380E166E050E00E94F90D2A
:1009F0004091850383E166E050E00E94F90D20916B
:100A0000BC01E199FECF89E190E09FBB8EBB2DBB7D
:100A10000FB6F894E29AE19A0FBE0AC0E199FECFB0
:100A200089E190E09FBB8EBBE09A8DB38093BC01BF
:100A30001F9108950E941E0383E66FE644E60E941C
:100A40008D1180E06CE40E94D0021092920180919E
:100A500092018823E1F387E062E040E750E00E94E2
:100A6000A00E0E945C061092920180919201882350
:100A7000E1F310929201809192018823E1F31092A8
:100A80009201809192018823E1F31092920180916A
:100A900092018823E1F310929201809192018823C0
:100AA000E1F31092920184E064E00E94D00280E0C1
:100AB0006CE40E94D00280919901882319F40E946D
:100AC00090041CC082E062E04CE751E00E94A00E5E
:100AD00082E064E042E951E00E94A00E82E066E01C
:100AE0004FE951E00E94A00EE199FECF89E190E02C
:100AF0009FBB8EBBE09A8DB38093BC018091920125
:100B00008823E1F310929201809192018823E1F30E
:100B10001092920184E064E00E94D00280E06CE4D4
:100B20000E94D00280919901882319F40E94350314
:100B300026C082E062E04CE351E00E94A00E82E019
:100B400064E043E551E00E94A00E82E066E040E6EA
:100B500051E00E94A00EE199FECF88E190E09FBB9A
:100B60008EBBE09A8DB38093C001E199FECF8AE1FC
:100B700090E09FBB8EBBE09A8DB38093090180917A
:100B8000BC01823029F483E66FE64AE00E948D11B1
:100B90008091BC01813029F482E664E64AE00E943B
:100BA0008D11809192018823E1F31092920180913E
:100BB00092018823E1F3109292018091920188239F
:100BC000E1F310929201809192018823E1F3109257
:100BD0009201809192018823E1F31092920184E0C6
:100BE00064E00E94D002089582E083BF82E48EBD5B
:100BF0008AE089BF08951F920F920FB60F921124B9
:100C00008F939F93809196018F5F8093960180913F
:100C10009601883449F591E09093950110929601E0
:100C20008091EA038F5F8093EA038091EA03843620
:100C300031F41092EA039093920190939301809182
:100C4000EA03823319F481E0809393018091E903F0
:100C50008F5F8093E9038091E9038A3029F4109231
:100C6000E90381E0809394019F918F910F900FBED3
:100C70000F901F901895982F80538A3010F020E025
:100C800005C0903311F42AE001C0282F892F815428
:100C90008A3110F4292F2653892F81568A3110F476
:100CA000292F2C539D3211F429E403C09E3209F4FC
:100CB00021E4822F0895089585E060E00E94D0022B
:100CC00086E063E80E94D00287E060E90E94D002DB
:100CD00085E060E00E94D00286E064E80E94D002D5
:100CE00087E061E90E94D00285E060E00E94D002C6
:100CF00086E065E80E94D00287E062E90E94D002A7
:100D000085E060E00E94D00286E066E80E94D002A2
:100D100087E063E90E94D00285E060E00E94D00293
:100D200086E067E80E94D00287E064E90E94D00272
:100D300085E060E00E94D00286E068E80E94D00270
:100D400087E065E90E94D00285E060E00E94D00261
:100D500086E069E80E94D00287E066E90E94D0023E
:100D600085E060E00E94D00286E06AE80E94D0023E
:100D700087E067E90E94D00285E060E00E94D0022F
:100D800086E061EA0E94D00287E068E90E94D00212
:100D900085E060E00E94D00286E062EA0E94D00214
:100DA00087E069E90E94D00285E060E00E94D002FD
:100DB00086E063EA0E94D00287E06AE90E94D002DE
:100DC00085E060E00E94D00286E064EA0E94D002E2
:100DD00087E06BE90E94D00285E060E00E94D002CB
:100DE00086E065EA0E94D00287E06CE90E94D002AA
:100DF00085E060E00E94D00286E066EA0E94D002B0
:100E000087E06DE90E94D00285E060E00E94D00298
:100E100086E067EA0E94D00287E06EE90E94D00275
:100E200085E060E00E94D00286E068EA0E94D0027D
:100E300087E06FE90E94D00285E060E00E94D00266
:100E400086E06FEB0E94D00287E060EA0E94D00249
:100E500085E060E00E94D00286E060EC0E94D00253
:100E600087E061EA0E94D00285E060E00E94D00243
:100E700086E061EC0E94D00287E062EA0E94D00224
:100E800085E060E00E94D00286E062EC0E94D00221
:100E900087E063EA0E94D00285E060E00E94D00211
:100EA00086E063EC0E94D00287E064EA0E94D002F0
:100EB00085E060E00E94D00286E064EC0E94D002EF
:100EC00087E065EA0E94D00285E060E00E94D002DF
:100ED00086E065EC0E94D00287E066EA0E94D002BC
:100EE00085E060E00E94D00286E066EC0E94D002BD
:100EF00087E067EA0E94D00285E060E00E94D002AD
:100F000086E06DED0E94D00287E068EA0E94D00280
:100F100085E060E00E94D00286E06EED0E94D00283
:100F200087E069EA0E94D00285E060E00E94D0027A
:100F300086E06FED0E94D00287E06AEA0E94D0024C
:100F400085E060E00E94D00286E060EE0E94D00260
:100F500087E06BEA0E94D00285E060E00E94D00248
:100F600086E061EE0E94D00287E06CEA0E94D00227
:100F700085E060E00E94D00286E062EE0E94D0022E
:100F800087E06DEA0E94D00285E060E00E94D00216
:100F900086E063EE0E94D00287E06EEA0E94D002F3
:100FA00085E060E00E94D00286E064EE0E94D002FC
:100FB00087E06FEA0E94D00285E060E00E94D002E4
:100FC00086E06BEF0E94D00287E060EB0E94D002C7
:100FD00085E060E00E94D00286E06CEF0E94D002C3
:100FE00087E061EB0E94D00285E060E00E94D002C1
:100FF00086E06DEF0E94D00287E062EB0E94D00293
:1010000085E060E00E94D00286E06EEF0E94D00290
:1010100087E063EB0E94D00285E060E00E94D0028E
:1010200086E06FEF0E94D00287E064EB0E94D0025E
:1010300085E061E00E94D00286E060E00E94D0027C
:1010400087E065EB0E94D00285E061E00E94D0025B
:1010500086E061E00E94D00287E066EB0E94D00249
:101060000895BF92CF92DF92EF92FF920F931F935A
:10107000CF93DF937C01B62E8C0145E0C42ED12C9A
:10108000C80ED91E862F90E0EC01CC0FDD1FC80FD3
:10109000D91FCA5EDE4F0EC085E0612F0E94D002CC
:1010A00086E0602F0E94D00287E068810E94D00213
:1010B0000F5F1F4F0C151D0578F38701065F1F4F4B
:1010C0008FE090E0E80EF91E8B2D90E0EC01CC0F44
:1010D000DD1FC80FD91FCA5EDE4F0EC085E0612F2D
:1010E0000E94D00286E0602F0E94D00287E06881D3
:1010F0000E94D0020F5F1F4F0E151F0578F3DF917E
:10110000CF911F910F91FF90EF90DF90CF90BF9004
:101110000895EF92FF920F931F93CF93DF938C016B
:10112000EC0155E0E52EF12CE80EF91E0DC085E02E
:101130006D2F0E94D00286E06C2F0E94D00287E0C3
:1011400060E00E94D0022196CE15DF0580F3E80111
:101150002A96015F1F4F0DC085E06D2F0E94D002BF
:1011600086E06C2F0E94D00287E060E00E94D002EF
:101170002196C017D10780F3DF91CF911F910F9176
:10118000FF90EF9008951F93CF93DF93C091470294
:10119000D0914802D7FD12C0CE016AE070E00E94F3
:1011A000761C182F16952091040130E0CE016AE0DC
:1011B00070E00E94761C261B310918C0EE27FF271D
:1011C000EC1BFD0BCF016AE070E00E94761C182F2B
:1011D00016951C5F2091040130E02F5F3F4FCF0137
:1011E0006AE070E00E94761C260F311DE90175E06F
:1011F000CC0FDD1F7A95E1F7220F331FC21BD30BF3
:1012000027968091120190911301C817D90739F0E0
:1012100080911201909113010E94890804C080916D
:10122000C901811721F0CE01612F0E94310810936E
:10123000C901D0931301C0931201DF91CF911F9187
:101240000895CF92DF92EF92FF920F931F93CF9367
:10125000DF938C01E62E85E0612F0E94D00286E0AC
:10126000602F0E94D002CE2CDD2484E391E0C80ED2
:10127000D91E87E0F60160810E94D002EEE1EE2ED9
:10128000F12CE00EF11E85E06F2D0E94D00286E069
:101290006E2D0E94D00287E0F60160810E94D0028C
:1012A000E801CC54DF4F025F1E4F85E06D2F0E9496
:1012B000D00286E06C2F0E94D00287E0F6016081A8
:1012C0000E94D0026E96C017D10779F7DF91CF91B7
:1012D0001F910F91FF90EF90DF90CF900895EF92C4
:1012E000FF920F931F93CF93DF937C0185E06F2DC7
:1012F0000E94D00286E06E2D0E94D00287E060E05E
:101300000E94D0028701025E1F4F85E0612F0E947C
:10131000D00286E0602F0E94D00287E060E00E9449
:10132000D002E701CC54DF4F8701025F1E4F85E0FA
:101330006D2F0E94D00286E06C2F0E94D00287E0C1
:1013400060E00E94D0026E96C017D10781F7DF914E
:10135000CF911F910F91FF90EF9008951F93CF931E
:10136000DF93E0914502F0914602F7FD14C0CF01F2
:101370006AE070E00E94761C182F16951C5F809121
:101380000501C82FD0E0CF016AE070E00E94761C12
:10139000C61BD10917C0222733272E1B3F0BC901BB
:1013A0006AE070E00E94761C182F16958091050166
:1013B000C82FD0E02196C9016AE070E00E94761C37
:1013C000C60FD11D8091140190911501C817D9073E
:1013D00039F080911401909115010E946F0904C0A9
:1013E0008091CA01811721F0CE01612F0E9421094D
:1013F0001093CA01D0931501C0931401DF91CF91CE
:101400001F91089585E060E00E94D00286E06FECB5
:101410000E94D00287E06CE80E94D00285E061E083
:101420000E94D00286E06BE00E94D00287E06DE867
:101430000E94D0020895EF92FF920F931F93CF93D3
:10144000DF937A019EE1699FB0011124680F711D3D
:101450008B01020F111D1092EB03EB0115C085E00B
:101460006D2F0E94D00286E06C2F0E94D0028091E6
:10147000EB03F701E80FF11D60818F5F8093EB03B1
:1014800087E00E94D0022196C017D10740F3DF9178
:10149000CF911F910F91FF90EF90089560910301FC
:1014A00081E04DE051E025E00E941B0A0895DF93A2
:1014B000CF9300D000D0CDB7DEB7F89430914D0275
:1014C0007894832F6AE00E94491C282F0E94491CAF
:1014D000482F822F0E94491C292F832F0E94491CCC
:1014E000992319F48AE08C8301C09C83222319F488
:1014F0008AE08A8301C02A83498385E48B8383E061
:1015000061E0AE014F5F5F4F24E00E941B0A0F9025
:101510000F900F900F90CF91DF910895DF93CF93AD
:1015200000D000D0CDB7DEB780E289839BE09A83FC
:1015300081E38B839C8381E061E0AE014F5F5F4F6D
:1015400021E00E941B0A80919B01813079F462E0C6
:10155000AE014E5F5F4F21E00E941B0A81E063E015
:10156000AE014D5F5F4F22E00E941B0A0F900F906B
:101570000F900F90CF91DF910895DF93CF9300D01C
:1015800000D00F92CDB7DEB7DE011196E1E4F1E0B5
:1015900085E001900D928150E1F7609104018CE0AB
:1015A000AE014F5F5F4F25E00E941B0A0F900F9026
:1015B0000F900F900F90CF91DF91089580E06CE431
:1015C0000E94D00208958091570390915803843B64
:1015D000910554F08091D90390E02091550330910A
:1015E00056038217930744F08091CB01882371F44E
:1015F00081E08093CB0108958091CB01181624F4EB
:1016000080E06CE40E94D0021092CB01089580E04B
:1016100062E40E94D00208958F929F92AF92BF928F
:10162000CF92DF92EF92FF920F931F93DF93CF93AE
:10163000CDB7DEB72F970FB6F894DEBF0FBECDBF84
:10164000FE013B9685E0DF011D928A95E9F78091C6
:10165000490290914A026EE170E00E94761CCB0133
:10166000019797FF02C080E090E08E010F5F1F4F4F
:10167000B8014AE050E00E94101CF80101900020DF
:10168000E9F73197FE2EF01A80E0CF2CDD24C7FC5D
:10169000D094F6E08F2E912C8C0E9D1E58010BC01D
:1016A000F501E00FF11F80810E943B06080D191D16
:1016B000F80180838E2D082F10E0E82EE3940C159E
:1016C0001D0574F38093EB0385E169E0AE01455F8E
:1016D0005F4F25E00E941B0A89E18F1969E0A40190
:1016E0002F2D0E941B0A2F960FB6F894DEBF0FBE57
:1016F000CDBFCF91DF911F910F91FF90EF90DF90C1
:10170000CF90BF90AF909F908F9008958F929F92AF
:10171000AF92BF92CF92DF92EF92FF920F931F93FF
:10172000DF93CF93CDB7DEB72E970FB6F894DEBF19
:101730000FBECDBF19821A821B821C828091B0011C
:101740009091B1018E010B5F1F4FB8014AE050E04C
:101750000E94101CF80101900020E9F73197FE2E3D
:10176000F01A80E0CF2CDD24C7FCD094AAE08A2EAA
:10177000912C8C0E9D1E58010BC0F501E00FF11F3E
:1017800080810E943B06080D191DF80180838E2D73
:10179000082F10E0E82EE3940C151D0574F38093D8
:1017A000EB0385E166E0AE014F5F5F4F24E00E94EE
:1017B0001B0A89E18F1966E0A4012F2D0E941B0AE4
:1017C0008091B0019091B1011816190664F485E07A
:1017D00060E00E94D00286E062EC0E94D00287E0C6
:1017E0006CE80E94D0028091B0019091B10197FF06
:1017F0000CC085E060E00E94D00286E062EC0E94AE
:10180000D00287E06DE80E94D0028091B0019091F3
:10181000B101892B61F485E060E00E94D00286E08E
:1018200062EC0E94D00287E060E00E94D0022E9617
:101830000FB6F894DEBF0FBECDBFCF91DF911F91E1
:101840000F91FF90EF90DF90CF90BF90AF909F905F
:101850008F9008958F929F92AF92BF92CF92DF9216
:10186000EF92FF920F931F93DF93CF93CDB7DEB725
:101870002B970FB6F894DEBF0FBECDBFDE011196D9
:10188000EEE3F1E083E001900D928150E1F78E01EB
:101890000C5F1F4F8091530390915403B8014AE0AD
:1018A00050E00E94101CF80101900020E9F73197E8
:1018B000FE2EF01A80E0CF2CDD24C7FCD094B8E0D7
:1018C0008B2E912C8C0E9D1E58010BC0F501E00F44
:1018D000F11F80810E943B06080D191DF8018083CD
:1018E0008E2D082F10E0E82EE3940C151D0574F3DF
:1018F0008093EB038DE06EE0AE014F5F5F4F23E01E
:101900000E941B0A80E18F196EE0A4012F2D0E9416
:101910001B0A2B960FB6F894DEBF0FBECDBFCF913A
:10192000DF911F910F91FF90EF90DF90CF90BF90CC
:10193000AF909F908F9008958F929F92AF92BF9299
:10194000DF92EF92FF920F931F93DF93CF93CDB768
:10195000DEB728970FB6F894DEBF0FBECDBF198251
:101960008AE08A838091A2019091A3018E010D5F8C
:101970001F4FB8014AE050E00E94101CF80101908E
:101980000020E9F73197E01B80E0EE2EFF24E7FC12
:10199000F094480106E0A02EB12CAC0EBD1E0BC089
:1019A000F401E00FF11F80810E943B060A0D1B1D10
:1019B000F80180838D2D082F10E0D82ED3940E15BA
:1019C0001F0574F38093EB038091A2019091A30112
:1019D0008E010A5F1F4F0A977CF46091030181E03A
:1019E000AE014F5F5F4F21E00E941B0A609103012F
:1019F00082E0A80121E005C06091030181E0A80117
:101A000022E00E941B0A8091A4019091A5018E0101
:101A10000D5F1F4FB8014AE050E00E94101CF80112
:101A200001900020E9F73197E01B80E0EE2EFF24C3
:101A3000E7FCF094480116E0A12EB12CAC0EBD1EBF
:101A40000BC0F401E00FF11F80810E943B060A0DDC
:101A50001B1DF80180838D2D082F10E0D82ED39404
:101A60000E151F0574F38093EB038091A4019091F0
:101A7000A5018E010A5F1F4F0A977CF46091030154
:101A800084E0AE014E5F5F4F21E00E941B0A60912F
:101A9000030185E0A80121E005C06091030184E015
:101AA000A80122E00E941B0A28960FB6F894DEBF18
:101AB0000FBECDBFCF91DF911F910F91FF90EF909F
:101AC000DF90BF90AF909F908F9008950F931F93DA
:101AD000DF93CF93CDB7DEB72A970FB6F894DEBF6A
:101AE0000FBECDBF8E010F5F1F4FB8014AE050E01F
:101AF0000E94101CF80101900020E9F73197E01BCB
:101B000020E0FF27E7FDF095322F3F5F822F90E026
:101B10008E179F0714F4232FF7CF2093EB032A96F9
:101B20000FB6F894DEBF0FBECDBFCF91DF911F91EE
:101B30000F910895AF92BF92CF92DF92EF92FF92F2
:101B40000F931F93DF93CF93CDB7DEB76E970FB68A
:101B5000F894DEBF0FBECDBFB82EA62ED42EA42F74
:101B6000B52FFD0101900020E9F73197CE2EC41A60
:101B70007E010894E11CF11C242F352FC9018C0132
:101B800008C0F80181918F010E943B06F701819303
:101B90007F01802F8D198C15A0F38B2D6A2DAE013E
:101BA0004F5F5F4F2C2D0E941B0A6E960FB6F89464
:101BB000DEBF0FBECDBFCF91DF911F910F91FF9080
:101BC000EF90DF90CF90BF90AF90089580919A01F1
:101BD000813071F4609106012091E1013091E201C0
:101BE000369527958EE0821B43EE51E00E949A0DB8
:101BF0000895EF92FF920F931F93DF93CF93CDB78A
:101C0000DEB764970FB6F894DEBF0FBECDBFF82ED7
:101C1000E62ECA018E010F5F1F4FB8014AE050E067
:101C20000E94101C8F2D6E2DA8010E949A0D6496A3
:101C30000FB6F894DEBF0FBECDBFCF91DF911F91DD
:101C40000F91FF90EF900895EF92FF920F931F93E3
:101C5000DF93CF93CDB7DEB72A970FB6F894DEBFE8
:101C60000FBECDBF20919203822F6AE00E94551CC7
:101C7000382F822F6AE00E94551C85E48F83809163
:101C80009303882309F48AE08887992319F48AE06A
:101C90008E8301C09E833D8319821A821B821C821F
:101CA00083E062E0AE014B5F5F4F24E00E941B0ABD
:101CB00080919603909197038952934234F088E281
:101CC00093E290939703809396038091960390916B
:101CD000970397FF04C010929703109296038E010A
:101CE0000B5F1F4F8091960390919703B8014AE0D4
:101CF00050E00E94101CF80101900020E9F77F01DC
:101D00000894E108F108E01AF10A83E063E0AE010B
:101D10004F5F5F4F24E00E941B0A87E08E1963E04B
:101D2000A8010E949A0D2A960FB6F894DEBF0FBE46
:101D3000CDBFCF91DF911F910F91FF90EF9008954C
:101D4000BF92CF92DF92EF92FF920F931F93DF9398
:101D5000CF93CDB7DEB764970FB6F894DEBF0FBE52
:101D6000CDBFC82EB62EFA017E010894E11CF11CED
:101D700004C0AE0DBF1D9C9331968E2F841B949191
:101D8000A82FB0E09923A9F7AE0DBF1D1C92F70153
:101D900001900020E9F73197DE2EDE18870107C099
:101DA000F80180810E943B06F80181938F01802F0A
:101DB0008E198D15A8F38C2D6B2DAE014F5F5F4FE3
:101DC0002D2D0E941B0A64960FB6F894DEBF0FBE3D
:101DD000CDBFCF91DF911F910F91FF90EF90DF90DA
:101DE000CF90BF9008951F93CF93DF93EC01A3E0B2
:101DF000B0E047C0FD01E758FD4F8081FD01E65886
:101E0000FD4F2081422F50E04D535040FD01E558D9
:101E1000FD4F7081FD01E458FD4F10819A01F4E0FF
:101E200035952795FA95E1F790E0CD97880F991FA2
:101E3000880F991F282B392B2883613029F1E72F30
:101E4000F0E0FD9734E0440F551F3A95E1F75070EC
:101E5000CF019595879595958795482B592B498363
:101E6000623091F01496635086E0EE0FFF1F8A9562
:101E7000E1F7F070812F90E0CD97E82BF92BEA8302
:101E80002396662309F0B6CFDF91CF911F91089575
:101E900080917B028635B1F480917A0281568093DD
:101EA000BC018091BC01843018F084E08093BC01B7
:101EB00083E893E06AE043E02AE00E94F30E81E0C9
:101EC0008093BD011092970108951F931091BC015A
:101ED000123009F474C0143009F4C9C0113009F08B
:101EE00089C180917B02813581F48FEB93E062E3BD
:101EF00043E02DE20E94F30E8091BF0390E09093A7
:101F0000BF018093BE011093C20180917B02843493
:101F100009F070C181E493E061E443E021E40E94B0
:101F2000F30E8091570390915803843B91053CF444
:101F300080919C01813051F410929C0107C08091E6
:101F40009C01882319F481E080939C0180914303D4
:101F50009091440365EF7FEF0E94761C6E5F7F4F88
:101F60007093480260934702809145039091460325
:101F70006BE070E00E94761C6A5F7F4F70934602B0
:101F80006093450280914D0390914E0390934A02D5
:101F9000809349028091550380934D0280912C02D9
:101FA00090912D0290934C0280934B0280915303A9
:101FB000909154039093500280934F021BC18091E3
:101FC0007B028F34A9F0813509F014C18FEB93E0C7
:101FD00062E343E02DE20E94F30E8091BF0390E0A4
:101FE0009093BF018093BE0181E08093C20102C142
:101FF00087EF91E060E543E02DE20E94F30E8091CF
:102000003702992787FD9095029690934802809316
:10201000470280913802992787FD90950696909304
:1020200046028093450280912A0290912B02909360
:102030004A02809349028091300280934D02809140
:102040002C0290912D0290934C0280934B02809130
:102050003502909136029093500280934F02809106
:1020600029028093510281E08093C101C3C0809115
:102070007B02843409F05AC081E493E061E443E0D8
:1020800021E40E94F30E8091570390915803843B02
:10209000910554F480919C01813031F410929C019F
:1020A000F8940E940E1178948091570390915803F0
:1020B000843B91057CF080919C01882359F481E058
:1020C00080939C01F89480919901882311F40E94D7
:1020D000FE107894809143039091440366E170E090
:1020E0000E94761C6E5F7F4F709348026093470298
:1020F000809145039091460366E170E00E94761C52
:102100006A5F7F4F709346026093450280914D0352
:1021100090914E0390934A02809349028091530319
:10212000909154039093500280934F0280917B02D0
:102130008C3481F481E090E09093BF018093BE01E4
:1021400081E08093C20181EC93E069E143E02DE2FC
:102150000E94F30E80917B028D3481F482E090E046
:102160009093BF018093BE0181E08093C20181EC16
:1021700093E069E143E02DE20E94F30E80917B023F
:102180008E3481F483E090E09093BF018093BE0190
:1021900081E08093C20181EC93E069E143E02DE2AC
:1021A0000E94F30E80917B028F3481F484E090E0F2
:1021B0009093BF018093BE0181E08093C20181ECC6
:1021C00093E069E143E02DE20E94F30E80917B02EF
:1021D000803581F485E090E09093BF018093BE014B
:1021E00081E08093C20181EC93E069E143E02DE25C
:1021F0000E94F30E109297011F91089582E289B90F
:1022000010BC80B91CBE909A28E92AB996E890BD06
:1022100082EC8BB921B99CBF82B9089582E289B959
:1022200010BC80B91CBE88E98AB926E820BD92ECB2
:102230009BB980E981B92CBF92B90895DF93CF9300
:10224000CDB7DEB72C970FB6F894DEBF0FBECDBF6B
:1022500083E2898383E68A8385E78B838DE38C839E
:102260008D838E838F83DE011196FD0120E030E0A7
:10227000AE01485F5F4F8191280F311DE417F507CC
:10228000D1F7C9019F7046E0959587954A95E1F78A
:10229000835C88872F733070822F835C89878DE001
:1022A0008A879E01255F3F4F8C91159BFECF83B996
:1022B0001196A217B307C1F72C960FB6F894DEBF9C
:1022C0000FBECDBFCF91DF910895DF93CF93CDB7F0
:1022D000DEB72C970FB6F894DEBF0FBECDBF8BE1F3
:1022E00089838A8385E58B838AEA8C831D82FE013C
:1022F00031969E012A5F3F4F8081159BFECF83B9A7
:102300003196E217F307C1F72C960FB6F894DEBFAB
:102310000FBECDBFCF91DF910895DF93CF93CDB79F
:10232000DEB72A970FB6F894DEBF0FBECDBF93E29B
:1023300099838A836B83842F86958695835C8C83AF
:1023400050E04370507064E0440F551F6A95E1F708
:10235000435C4D838DE38E838F83DE011196FD01F7
:1023600020E030E0AE01485F5F4F8191280F311DC2
:10237000E417F507D1F7C9019F7056E09595879549
:102380005A95E1F7835C88872F733070822F835CC6
:1023900089878DE08A879E01255F3F4F8C91159B31
:1023A000FECF83B91196A217B307C1F72A960FB6CD
:1023B000F894DEBF0FBECDBFCF91DF9108955D9B36
:1023C000FECF8DE68CB95D9BFECF8FE68CB95D9B11
:1023D000FECF89E68CB95D9BFECF8EE68CB95D9B06
:1023E000FECF8DE08CB95D9BFECF8EE38CB9089556
:1023F000982F9F7082958F708A3010F4805D01C095
:10240000895C5D9BFECF8CB99A3018F4892F805D72
:1024100002C0892F895C5D9BFECF8CB908958A30FC
:1024200010F4805D01C0895C5D9BFECF8CB908957E
:10243000159BFECF83B908955D9BFECF8CB908959F
:10244000662359F020E0FC01E20FF11DE0815D9B65
:10245000FECFECB92F5F6217B0F708955D9BFECFFA
:102460008EE38CB908951F920F920FB60F9211242C
:102470002F933F938F939F93AF93BF93EF93FF93CC
:102480002CB12093EC0385B398E0892785BB5D9B35
:10249000FECF2CB92D3059F08091BE03E82FF0E02B
:1024A000E856FC4F20838F5F8093BE035FC0E091AE
:1024B000BE03F0E0E856FC4F20831092B901109261
:1024C000BA011092BB0130E020E090E045C021301D
:1024D000B9F0213018F02230F1F528C0A32FB0E078
:1024E000A856BC4F8C91803211F421E033C0E92F03
:1024F000F0E08C91EA54FC4F80839093B9010FC0B7
:10250000A32FB0E0A856BC4F8C91E92FF0E08032A9
:1025100041F08C91E459FD4F80839093BA019F5F05
:102520001AC0E459FD4F108222E014C0A32FB0E07E
:10253000A856BC4F8C91E92FF0E08D3039F08C918A
:10254000ED5AFD4F80839093BB01E9CFED5AFD4FCB
:10255000108223E090E03F5F8091BE03831708F074
:10256000B6CF81E08093B8011092BE03FF91EF9146
:10257000BF91AF919F918F913F912F910F900FBE7F
:102580000F901F9018951F920F920FB60F92112463
:102590008F939F93EF93FF9393B19093ED039D30AF
:1025A00081F48091CC01813061F4AB981092CC0120
:1025B00080939701E0918E03F0E0E758FD4F908300
:1025C0002DC08091CC01882319F0813039F514C0D9
:1025D000933241F480919701882321F481E0809324
:1025E000CC01AB9A10928E0380918E03E82FF0E01D
:1025F000E758FD4F90830CC0E0918E03F0E0E75860
:10260000FD4F908380918E03873C30F480918E0340
:102610008F5F80938E0302C01092CC01FF91EF91E7
:102620009F918F910F900FBE0F901F90189585B3BB
:1026300092E0892785BB089590919F01913019F40C
:1026400085B3892785BB08951F920F920FB60F920D
:1026500011242F933F935F936F937F938F939F9357
:10266000AF93BF938091CE019091CF01892B81F4DC
:1026700084B595B59093D5018093D4018EB58F7BA9
:102680008EBD81E090E09093CF018093CE013AC05F
:1026900084B595B59093D3018093D2012EB5206473
:1026A0002EBD2091D4013091D5011092CF0110920E
:1026B000CE01821B930B865698406CE271E00E941B
:1026C000621C7093D1016093D0016730710534F0C2
:1026D00086E090E09093D1018093D0012091D001C9
:1026E0003091D10180910201992787FD909528179B
:1026F000390741F0263031052CF42093020181E0A6
:102700008093A601BF91AF919F918F917F916F911F
:102710005F913F912F910F900FBE0F901F901895D2
:102720008091490290914A029093A9018093A80157
:102730008091A8019091A9012091AA013091AB014B
:10274000821B930B9093AD018093AC018091A80103
:102750009091A9019093AB018093AA014091B4019B
:102760005091B5018091AC019091AD01E3E0880FEB
:10277000991FEA95E1F79A0173E0220F331F7A95CA
:10278000E1F7241B350B820F931F68E070E00E9475
:10279000761C7093B5016093B4012091B60130911D
:1027A000B7014091B4015091B501C90163E0880FB0
:1027B000991F6A95E1F7821B930B840F951F68E0C0
:1027C00070E00E94761C7093B7016093B60180910F
:1027D000B6019091B7019093B1018093B0010E942E
:1027E000860B0895609104018BE14EE451E00E9454
:1027F0009A0D80913B0281FF07C0609104018BE13B
:1028000041E551E00E949A0D80913B0282FF07C092
:10281000609104018BE144E551E00E949A0D089516
:10282000DF93CF930F92CDB7DEB7809125029091C1
:10283000260221E0823592071CF080EC898307C0D4
:102840004E966DE270E00E94761C60546983609140
:1028500004018EE0AE014F5F5F4F21E00E941B0A32
:102860000F90CF91DF9108958AE161E047E551E053
:1028700022E00E941B0A0895DF93CF9300D000D07E
:10288000CDB7DEB719821A821B821C8260910301C8
:10289000615085E1AE014F5F5F4F24E00E941B0A4B
:1028A000609103016150409112025091130285E141
:1028B0000E94F90D0F900F900F900F90CF91DF9124
:1028C0000895DF93CF9300D00F92CDB7DEB7DE012E
:1028D0001196E9E5F1E083E001900D928150E1F776
:1028E000609104016F5F8EE0AE014F5F5F4F23E0A8
:1028F0000E941B0A209104012F5F80912302909176
:1029000024026AE070E00E94761CAB018EE0622F28
:102910000E94F90D0F900F900F90CF91DF910895C5
:102920008F929F92BF92CF92DF92EF92FF920F937E
:102930001F93DF93CF93CDB7DEB72B970FB6F894E5
:10294000DEBF0FBECDBFDE011196ECE5F1E083E006
:1029500001900D928150E1F7809151028E010C5F40
:102960001F4F90E0B8014AE050E00E94101CF801AF
:1029700001900020E9F73197BE2EB01AEE24FF2413
:10298000CB2CDD24C7FCD09488E0882E912C8C0EB3
:102990009D1E0DC0F801EE0DFF1D80810E943B06BB
:1029A000F401EE0DFF1D80830894E11CF11CEC1472
:1029B000FD0484F388E161E0AE014F5F5F4F23E0E7
:1029C0000E941B0A8BE18B1961E0A4012B2D0E9450
:1029D0001B0A2B960FB6F894DEBF0FBECDBFCF916A
:1029E000DF911F910F91FF90EF90DF90CF90BF90FC
:1029F0009F908F9008958F929F92BF92CF92DF9277
:102A0000EF92FF920F931F93DF93CF93CDB7DEB773
:102A10006A970FB6F894DEBF0FBECDBFFE013196A8
:102A200086E0DF011D928A95E9F72091310230910D
:102A30003202C90143E0880F991F4A95E1F7820FDE
:102A4000931F6AEF70E00E94621CCB018E01095F48
:102A50001F4FB8014AE050E00E94101CF80101909D
:102A60000020E9F73197BE2EB01AEE24FF24CB2CBC
:102A7000DD24C7FCD09491E1892E912C8C0E9D1EF3
:102A80000DC0F801EE0DFF1D80810E943B06F40190
:102A9000EE0DFF1D80830894E11CF11CEC14FD0475
:102AA00084F36091030185E1AE014F5F5F4F26E043
:102AB0000E941B0A609103018BE18B19A4012B2D4D
:102AC0000E941B0A6A960FB6F894DEBF0FBECDBFF8
:102AD000CF91DF911F910F91FF90EF90DF90CF90FA
:102AE000BF909F908F90089583E66FE644E60E9422
:102AF0008D11F89428E088E190E00FB6F894A8953D
:102B000081BD0FBE21BDFFCF1F939D998AC18091CA
:102B1000D6018F5F8093D60111E01093D801809188
:102B2000D601853009F081C18091DA01882309F04E
:102B30008CC01093DA011092DB0184E064E00E9403
:102B4000D00283E061E043EE51E00E949A0D83E001
:102B500063E040E152E00E94A00E84E068E00E9441
:102B6000D00283E065E049E152E00E94A00E80912E
:102B70000001813029F484E165E045E452E004C0BD
:102B800084E165E048E452E00E94A00E84E060E049
:102B90000E94D00283E066E04DE152E00E94A00E68
:102BA00080919901813029F484E166E045E452E0A6
:102BB00004C084E166E048E452E00E94A00E83E095
:102BC00067E043E252E00E94A00E80919A018130BA
:102BD00029F484E167E045E452E004C084E167E061
:102BE00048E452E00E94A00E83E068E04BE252E02D
:102BF0000E94A00E8091A701813029F484E168E051
:102C000045E452E004C084E168E048E452E00E94F8
:102C1000A00E83E069E046E352E00E94A00E80919E
:102C20009B01813029F484E169E045E452E004C06D
:102C300084E169E048E452E00E94A00E83E06BE08A
:102C400040E452E00E94A00EEEC08091DB01882398
:102C500049F584E068E00E94D00280910001882359
:102C600039F41093000184E165E045E452E006C0C8
:102C70001092000184E165E048E452E00E94A00E59
:102C800020910001E199FECF81E090E09FBB8EBBD7
:102C90002DBB0FB6F894E29AE19A0FBE84E060E093
:102CA0000E94D0021091DB01113049F584E068E008
:102CB0000E94D00280919901882339F410939901E0
:102CC00084E166E045E452E006C01092990184E197
:102CD00066E048E452E00E94A00E20919901E1993B
:102CE000FECF80E090E09FBB8EBB2DBB0FB6F8946B
:102CF000E29AE19A0FBE84E060E00E94D0028091E7
:102D0000DB01823051F584E068E00E94D0028091BE
:102D10009A01882341F481E080939A0184E167E07D
:102D200045E452E006C010929A0184E167E048E46D
:102D300052E00E94A00E20919A01E199FECF82E01C
:102D400090E09FBB8EBB2DBB0FB6F894E29AE19A40
:102D50000FBE84E060E00E94D0028091DB018330EE
:102D600051F584E068E00E94D0028091A701882399
:102D700041F481E08093A70184E168E045E452E0FA
:102D800006C01092A70184E168E048E452E00E9486
:102D9000A00E2091A701E199FECF87E190E09FBBB3
:102DA0008EBB2DBB0FB6F894E29AE19A0FBE84E079
:102DB00060E00E94D0028091DB01843049F568E038
:102DC0000E94D00280919B01882341F481E080938E
:102DD0009B0184E169E045E452E006C010929B014A
:102DE00084E169E048E452E00E94A00E20919B013A
:102DF000E199FECF8BE190E09FBB8EBB2DBB0FB660
:102E0000F894E29AE19A0FBE84E060E00E94D0025A
:102E10008091DB01853049F41092DA010E9474152B
:102E200004C01092D6011092D8019C9913C19091C0
:102E3000DA01913009F014C19093D9018091D70142
:102E40008F5F8093D7012091D701253009F008C109
:102E50001092D7018091DB01823009F469C0833080
:102E600030F4882371F0813009F0FAC035C0843025
:102E700009F4AAC0843008F486C0853009F0F0C097
:102E8000C3C09093DB0183E065E049E152E00E941A
:102E9000A00E80910001813029F484E165E045E4D1
:102EA00052E004C084E165E048E452E00E94A00ED4
:102EB00084E068E00E94D00283E066E04DE152E0E9
:102EC0000E94A00E80919901813019F484E166E09E
:102ED000B3C084E166E0B5C082E08093DB0183E0AB
:102EE00066E04DE152E00E94A00E80919901813090
:102EF00029F484E166E045E452E004C084E166E040
:102F000048E452E00E94A00E84E068E00E94D002F3
:102F100083E067E043E252E00E94A00E80919A01B4
:102F2000813019F484E167E087C084E167E089C0FB
:102F300083E08093DB0167E043E252E00E94A00E51
:102F400080919A01813029F484E167E045E452E000
:102F500004C084E167E048E452E00E94A00E84E0EF
:102F600068E00E94D00283E068E04BE252E00E94F9
:102F7000A00E8091A701813019F484E168E05CC063
:102F800084E168E05EC084E08093DB0183E068E078
:102F90004BE252E00E94A00E8091A701813029F4FB
:102FA00084E168E045E452E004C084E168E048E47C
:102FB00052E00E94A00E84E068E00E94D00283E00C
:102FC00069E046E352E03FC02093DB0183E069E023
:102FD00046E352E00E94A00E80919B01813029F4CB
:102FE00084E169E045E452E004C084E169E048E43A
:102FF00052E00E94A00E84E068E00E94D00283E0CC
:103000006BE040E452E01FC01092DB0183E06BE014
:1030100040E452E00E94A00E84E068E00E94D002EA
:1030200083E065E049E152E00E94A00E809100013A
:10303000813029F484E165E045E452E004C084E194
:1030400065E048E452E00E94A00E84E060E00E9447
:10305000D00206C01092D7018091D8018091D90189
:103060001F910895813061F4E199FECF80E090E0F6
:103070009FBB8EBB6DBB0FB6F894E29AE19A0FBE70
:103080000895DF93CF93CDB7DEB764970FB6F8946A
:10309000DEBF0FBECDBF20E0DE011196E199FECF6D
:1030A000E22FF0E0CF018D5F9F4F9FBB8EBBE09A78
:1030B0008DB3EA0FFB1F8083882311F02F5FEECFC3
:1030C000FD0101900020E9F79F01215030402A1BAB
:1030D0003B0B3093E2012093E10190E0AE014F5FA2
:1030E0005F4F09C0FD01ED51FE4FA40FB51F8C913C
:1030F000808311829F5FA92FB0E0A217B30790F3DE
:1031000064960FB6F894DEBF0FBECDBFCF91DF91AE
:103110000895DF93CF93CDB7DEB760970FB6F894DD
:10312000DEBF0FBECDBF80914F02909150029093B1
:1031300078028093770280917702909178026FE015
:1031400070E00E94621CDE011596AD016A1B9E01B3
:10315000205F3F4FE62FEA0FF0E0E55BFD4FE49183
:10316000ED93A217B307B1F76091070119821A8294
:103170001B821C8289E02BE00E941B0A60910801DF
:103180008EE0AE014F5F5F4F24E00E941B0A60910A
:10319000080140917702509178028FE00E94F90D6A
:1031A00060960FB6F894DEBF0FBECDBFCF91DF9112
:1031B0000895FF920F931F93DF93CF93CDB7DEB7A0
:1031C000E4970FB6F894DEBF0FBECDBFDE011C96AC
:1031D000EFE5F1E087E001900D928150E1F7DE012B
:1031E0005396E6E6F1E089E001900D928150E1F717
:1031F000DE019796EFE6F1E08EE001900D928150AE
:10320000E1F7DE011696EDE7F1E086E001900D9220
:103210008150E1F7DE015C96E3E8F1E08BE001909C
:103220000D928150E1F78091B6039091B7038734F6
:1032300009F066C0943409F063C080916C029091EB
:103240006D02813409F05CC09C3409F059C0E199E9
:10325000FECF81E090E09FBB8EBBE09A2DB32111A1
:1032600021E0022FE199FECF80E090E09FBB8EBB72
:10327000E09A8DB3882311F0022F0260E199FECF0E
:1032800082E090E09FBB8EBBE09A8DB38111046019
:10329000E199FECF87E190E09FBB8EBBE09A8DB3B2
:1032A00081110860E199FECF8BE190E09FBB8EBB5E
:1032B000E09A8DB38111006183E20E941C12802F7D
:1032C00090E08E010F5F1F4FB8014AE050E00E946E
:1032D000101CF80101900020E9F73197E01BF10B79
:1032E000C8016E2F0E9420128CE20E941C1283EEF5
:1032F00091E06091E1010E9420128DE00E941C1279
:103300008091B6039091B703833509F0B6C0943429
:1033100009F0B3C08CE692E00E94EB1BF82E03EE9E
:1033200011E0C80163E572E00E94091CD8010D900C
:103330000020E9F71197A01BB10B80E011C0F90143
:10334000ED51FE4FE081E199FECF2D5F3F4F3FBB36
:103350002EBBEDBB0FB6F894E29AE19A0FBE8F5FD9
:10336000282F30E02A173B0750F3E199FECF8F5FFB
:1033700090E08D5F9F4F9FBB8EBB1DBA0FB6F89438
:10338000E29AE19A0FBEB093E201A093E1012F2DE2
:10339000F0FE09C0E199FECF81E090E09FBB8EBBBB
:1033A00081E08DBB07C0E199FECF81E090E09FBB3B
:1033B0008EBB1DBA0FB6F894E29AE19A0FBE21FFB8
:1033C00009C0E199FECF80E090E09FBB8EBB81E019
:1033D0008DBB07C0E199FECF80E090E09FBB8EBB24
:1033E0001DBA0FB6F894E29AE19A0FBE22FF09C007
:1033F000E199FECF82E090E09FBB8EBB81E08DBB68
:1034000007C0E199FECF82E090E09FBB8EBB1DBA62
:103410000FB6F894E29AE19A0FBE23FF09C0E19932
:10342000FECF87E190E09FBB8EBB81E08DBB07C0E4
:10343000E199FECF87E190E09FBB8EBB1DBA0FB62E
:10344000F894E29AE19A0FBE24FF09C0E199FECFF9
:103450008BE190E09FBB8EBB81E08DBB07C0E19903
:10346000FECF8BE190E09FBB8EBB1DBA0FB6F894E8
:10347000E29AE19A0FBE0E9474155091B6036091D2
:10348000B7034091B8038091B90320E030E0803762
:1034900011F421E030E080E090E04C3611F481E05E
:1034A00090E02823392380E0583609F481E090E049
:1034B000653609F491E0892390E028233923232BF2
:1034C00079F0CE010C9666E00E942012CE01439660
:1034D00068E00E942012CE0187966DE00E942012C3
:1034E0005091B6036091B7034091B8038091B9033E
:1034F00020E030E0873711F421E030E080E090E018
:103500004F3611F481E090E02823392380E05337CF
:1035100009F481E090E0683609F491E0892390E0B5
:1035200028233923232B19F180916C0290916D028D
:10353000893481F4943471F4CE01069665E00E94DA
:10354000201283EE91E06091E1010E9420128DE053
:103550000E941C1280916C0290916D02863739F4A2
:10356000953629F4CE014C966CE00E942012809191
:10357000B6032091B7034091B80390E0833709F474
:1035800091E080E0253609F481E09823892F90E0CE
:1035900020E030E0443711F421E030E0822393232F
:1035A000892B09F442C080916C0290916D0289349C
:1035B00009F03BC0943409F038C020E01AC0FD0186
:1035C000ED5AFD4FE081E199FECF822F90E08D5FB3
:1035D0009F4F9FBB8EBBEDBB0FB6F894E29AE19A6A
:1035E0000FBEFD01ED5AFD4F8081AD51BE4F8C9352
:1035F0002F5F8091BB01A22FB0E0281700F3E19963
:10360000FECFCD018D5F9F4F9FBB8EBB1DBA0FB606
:10361000F894E29AE19A0FBEE22FF0E0ED51FE4FEE
:103620001082B093E201A093E1015091B603609142
:10363000B7034091B8038091B90320E030E08536AC
:1036400011F421E030E080E090E0433711F481E0B4
:1036500090E02823392380E0523709F481E090E09C
:10366000653609F491E0892390E028233923232B40
:1036700011F00E947415E4960FB6F894DEBF0FBEE9
:10368000CDBFCF91DF911F910F91FF9008951F92B1
:103690000F920FB60F9211242F933F938F939F9306
:1036A000EF93FF938091DD01882381F08091DD010C
:1036B00090E00197E0919001F0919101E80FF91FDE
:1036C0008FB1808381E08093DE0103C08FB180934E
:1036D000F3032091DD0180918E0130E0992787FD71
:1036E0009095821793075CF084E080938F0181E0CE
:1036F0008093DE018091DD018093F20308C0929AED
:103700001092DC0181E08093DF011092E001809152
:10371000DD018F5F8093DD01FF91EF919F918F918C
:103720003F912F910F900FBE0F901F90189582ED33
:103730008DB90895813029F4613011F4929808957B
:10374000929A0895982F8091DC018823C9F49130D2
:1037500009F492989093DC0181E08093E00191302C
:1037600069F486E080938E011092DD018AE08093F7
:103770008F019093DE018AEA8093F20380E008953E
:103780008091DE01813071F480918F0181508093AE
:103790008F018F5F39F48091F2038FB91092DE01AF
:1037A00081E0089581E00895CF93DF93C0E0D0E0F9
:1037B000E0919001F0919101EC0FFD1F80810E943A
:1037C000F8112196C730D10599F78DE00E941C129F
:1037D000DF91CF910895FC0188279927E8942191E2
:1037E0002032E9F3293010F02E30C8F32B3241F0AB
:1037F0002D3239F4689404C00E94311C820F911D4F
:10380000219120532A30C0F31EF4909581959F4F4B
:103810000895FB01DC0101900D920020E1F708956D
:10382000FB019F01E8944230C4F04532B4F44A30C1
:1038300029F497FB1EF4909581959F4F642F77276D
:103840000E94621C805D8A330CF0895D8193CB01FC
:103850000097A1F716F45DE251931082C9010C9410
:10386000391C7AE0979F902D879F802D910D112410
:103870000895DC01FC01672F71917723E1F73297FE
:1038800004C07C916D9370836291AE17BF07C8F33B
:103890000895991B79E004C0991F961708F0961BAC
:1038A000881F7A95C9F78095089587FB082E06260C
:1038B00087FD819567FD6195ECDF0EF4919507FC1E
:1038C00081950895AA1BBB1B51E107C0AA1FBB1F0E
:1038D000A617B70710F0A61BB70B881F991F5A959C
:1038E000A9F780959095BC01CD01089597FB092E0D
:1038F00007260AD077FD04D0E5DF06D000201AF4B1
:10390000709561957F4F0895F6F7909581959F4F3B
:063910000895F894FFCFBA
:103916000101030E0786010E0C5C00000A0000443C
:10392600000023002300546466536365526200510D
:1039360061005060005060005161005262005363A4
:10394600655464666768696A6B6B6A6968670000D4
:103956000053536353534103F701BF030D0A20205D
:10396600005048004348000A1D000000000000689F
:10397600656C70200D0073686F772049440D0073E5
:10398600686F772076657273696F6E0D0049442003
:103996003D2000302E392E342E302E310D000907F1
:0239A60091038B
:00000001FF
